:10243F00D2B4D2B5D2B6125A4920D803125A40128A
:10244F0059F812596F7839E6B45510C2B47F557EDA
:10245F00001255A775BF02783976AA1259887830BD
:10246F00A6077F017E001252027830E624EF601932
:10247F0024DE600924117016125A2E801C7FE77E0D
:10248F00001255A71259508010124E5E800B7830F3
:10249F00E6FF7E001255A7C2B47830E6D3940750FA
:1024AF00BAD2B41257877831A6071257877832A657
:1024BF00071257877833A6071257877834A6071263
:1024CF0057877835A6071257877836A6071257878A
:1024DF007837A6071257877838A60790F00AE49343
:1024EF00783AF67B007A007930751B0BE4FD7FF0AC
:0924FF001254C4124E5E0224487E
:100D02007830E614602F1460431460541460661443
:100D1200607A147003020DA124F57003020DAA2457
:100D2200116003020E131250057F1E7E0012520242
:100D32001250058021124D808F087E001255A7D2D5
:100D4200B5E508B4AA03020E0E020E13123C907F00
:100D5200017E001252027FAA7E001255A7020E0CDB
:100D62001225D01257878F08D2B5E508B4AA03021C
:100D72000E0E020E131246958F087E001255A7D250
:100D8200B5E508B4AA03020E0E020E1312120512E2
:100D920057878F08D2B5E508B4AA02806F80721215
:100DA20028D3C2B6D2B5806690F00AE493F5093032
:100DB200E00D1250057F1E7E00125202125005E510
:100DC2000930E118124D808F08E50864AA6002809C
:100DD20035C2B67F1E7E00125202D2B6E50930E25B
:100DE2000312349FE50930E30D1242488F08E508EB
:100DF20064AA60028010E50930E40F1246958F085C
:100E0200E50864AA6004D2B58007D2B5C2B6025A18
:060E120049C2B41259A010
:010E180022B7
:10500500125A0A7F017E00125202C2B57F047E0049
:10501500125202C2D97F0A7E0012520275905E00BA
:105025000000000000000000000000C2B200000007
:1050350000000000000000000075905F7FE87E031F
:10504500125202D2B2E4FFFE0000000000000FBFC2
:1050550000010EEF64144E70EFD2D97590FF7F01F9
:055065007E0002520272
:104D8000125A0A7F017E00125202C2B57F047E00D1
:104D9000125202C2D97F0A7E001252027590FF9011
:104DA000F004E493FFA3E493FE90F007E493FDA3E3
:104DB000E493FC8FA08E80D2DBC2DB7580FFC2B291
:104DC0000000C2B3000000000000AB800000000043
:104DD0000000D2B30000D2B2EBF460037F5522EFA3
:104DE000B50507EEB504037FAA220EEE70C50F804D
:014DF000C200
:103C9000125A0A7F017E00125202C2B57F047E00D2
:103CA000125202C2D97F0A7E001252027580FF9022
:103CB000F004E493F50AA3E493F50B90F007E49382
:103CC000F50CA3E493F50D850AA0850B80D2DBC229
:103CD000DB7580FF00001257878F807590570000BA
:103CE000C2B2000075905FE4FFFE0000000000001B
:103CF0000FBF00010EEF64044E70EFD2B2E50AB5BB
:103D00000C06E50B650D600A050BE50B70B9050A9D
:103D100080B5E4FEFF0000000000000FBF00010EB0
:063D2000EF641E4E70EF7F
:013D2600227A
:1025D000E4F510F50FF50EF50D125A0A7F017E0095
:1025E000125202C2B57F047E00125202C2D97F0A83
:1025F0007E001252027590FF90F004E493FBA3E476
:1026000093FA90F007E493F50AA3E493F98BA08A78
:1026100080D2DBC2DB7580FFC2B20000C2B3000013
:1026200000000000AF80000000000000D2B30000F6
:10263000D2B2E4FCFDFEE5102FF510EE350FF50FDC
:10264000ED350EF50EEC350DF50DEBB50A04EA6926
:1026500060070AEA70B70B80B4AF10AE0FAD0EACD6
:102660000D7810120A12AB07AF10AE0FAD0EAC0D05
:102670007808120A128F0BE510FFE48F0CAF03FEEF
:102680001255A7125787AF0B7E001255A712578716
:07269000AF0C7E000255A70C
:10469500125A0A7F0A7E00125202C2B57F047E00BA
:1046A500125202C2D97F0A7E001252027590CF00C3
:1046B5000000000000C2B20000000000007590DF9D
:1046C500E4FFFE0000000000000FBF00010EEF64D4
:1046D500324E70EFD2B2000000000000C2D9D2DA2B
:1046E5007590FFE4F5A0F580D2DBC2DB7580FFC2D3
:1046F500B20000C2B3000000000000AF800000005F
:10470500000000D2B30000D2B2EF60037F552275DE
:0447150090FF7FAAE8
:01471900227D
:1028D300E4F50FF510125A0A7F017E00125202C26C
:1028E300B57F047E00125202C2D9D2DA7F0A7E007B
:1028F3001252027590FF7834E6F50B08E6F50C7872
:1029030037E6F50D08E6F50E850BA0850C80D2DBC6
:10291300C2DB7580FFC2B20000C2B300000000003A
:102923000085800A000000000000D2B30000D2B28C
:10293300AF0A7E001255A70000000000000000004F
:102943000000000510E5107002050FB40026E50F26
:10295300B40221125787E50A6F600D7F557E00127E
:1029630055A7150B150B80077FAA7E001255A7E408
:10297300F50FF510E50BB50D06E50C650E600B05BF
:0A2983000CE50C7083050B02290B14
:01298D002227
:10120500E4F513F512F511F510F514F515125A0A52
:10121500C2B57834E6F50A08E6F50B7837E6F50C3D
:1012250008E6F50D75F65575F6AA75F65575BF0CF4
:10123500E4F5F475F7A275F7A205F405F40515E5CF
:1012450015700205146480451470E8850AF4850B51
:10125500F51257878FF675F7A0E50AFE7C00E425A1
:101265000BFFEC3E8F82F583E0FFE4FDFEE5132FD7
:10127500F513EE3512F512ED3511F511EC3510F5C6
:1012850010E50AB50C06E50B650D600A050BE50BC7
:1012950070B9050A80B575BF02AF13AE12AD11ACBA
:1012A500107810120A12AB07AF13AE12AD11AC10C5
:1012B5007808120A128F0EE513FFE48F0FAF03FEB5
:1012C5001255A7125787AF0E7E001255A7125787E2
:1012D500783AA6077B007A007930751B0BE4FD7F11
:0B12E500F01254C4AF0F7E000255A7AA
:10349F00125A0A7F017E00125202C2B57F047E00CB
:1034AF00125202C2D9D2DA7F0A7E001252027580FE
:1034BF00FF90F004E493FDA3E493FC90F007E493F2
:1034CF00F50AA3E493F98DA08C80D2DBC2DB758063
:1034DF00FF000075BF08EDFEEC7A002400FFEA3E06
:1034EF008F82F583E0F58075BF027590570000C29B
:1034FF00B2000075905FE4FFFE0000000000000FB7
:10350F00BF00010EEF64054E70EFD2B2EDB50A04A5
:10351F00EC6960070CEC70AE0D80ABE4FEFF0000B1
:0F352F00000000000FBF00010EEF64284E70EF88
:01353E00226A
:10424800750CAA125A0A7F017E00125202C2B57F6B
:10425800047E00125202C2D9D2DA7F0A7E001252BC
:10426800027590FF90F004E493FDA3E493FC90F0B2
:1042780007E493F50AA3E493F50B8DA08C80D2DBB9
:10428800C2DB7580FFC2B20000C2B30000000000AC
:1042980000A980000000000000D2B30000D2B2756F
:1042A800BF08EDFEEC7A002400FFEA3E8F82F5831A
:1042B800E075BF026960037F5522EDB50A07ECB5CA
:0C42C8000B037FAA220CEC70B10D80AE3D
:100526007830E614605514606E1470030205B21438
:1005360070030205CC1470030205E1147003020572
:10054600F924F570030206032411600302069712CC
:1005560059038F08E508B4AA0F12315E7F1E7E008C
:1005660012520212315E80397F1E7E001252027FC5
:10057600557E001255A7C2B40259B77F0A7E0012F3
:100586005202124BA38F087E001255A7D2B5E5087A
:10059600B4AA02802D80571232087F017E001252C3
:1005A600027FAA7E001255A7D2B5803E7F0A7E0042
:1005B600125202121C0B1257878F08D2B5E508B4E7
:1005C600AA0280268028123E518F087E001255A767
:1005D600D2B5E508B4AA02801180131212F01257A0
:1005E600878F08D2B5E508B4AA04C2B6800CC2B497
:1005F6000259A01230B0C2B6D2B5025A4990F00ADA
:10060600E493F50930E0231259038F08E50864AA3C
:100616006009D2B5C2B41259B7807B12315E7F1E13
:100626007E0012520212315ED2B5E50930E11F1288
:100636004BA38F08E50864AA6009D2B5C2B4125963
:10064600A08053C2B67F1E7E00125202D2B6E509C2
:1006560030E2031232B2E50930E3141249298F0859
:10066600E50864AA6009D2B5C2B41259A08027E58C
:100676000930E414123E518F08E50864AA6009D2D5
:10068600B5C2B41259A0800ED2B5C2B6125A49806C
:0906960005C2B41259A012596FFB
:01069F002238
:10315E0090F001E493FFBF4008750C00750D4080A0
:10316E0006750C00750D08125A0A7F017E00125268
:10317E0002C2B5C2D9D2DA7F0A7E00125202D2B38F
:10318E00759078C2B27590787590707590507F0179
:10319E007E00125202E4F50AF50BC3E50B950DE520
:1031AE000A950C501E7590517F067E0012520275C4
:1031BE0090507F017E00125202050BE50B70DB056D
:1031CE000A80D77F067E0012520275905800007555
:1031DE0090787F017E00125202D2B2E4FFFE000010
:1031EE00000000000FBF00010EEF64144E70EFD20E
:0A31FE00D9D2DA7F017E00025202EE
:104BA300750AAA125A0A7F017E00125202C2B5D2B6
:104BB300D9D2DA7F0A7E001252027590FF90F00478
:104BC300E493FFA3E493FE90F007E493FDA3E4933F
:104BD300FC8FA08E80D2DBC2DB7580FF000000005B
:104BE30000007590F80000C2B2C2B30000000000DC
:104BF30000AB80000000000000000000000000D2B5
:104C0300B3D2B2EBF460037F5522EFB50507EEB5DF
:0C4C130004037FAA220EEE70B80F80B5DB
:10320800125A0A7F017E00125202C2B57F047E0064
:10321800125202C2D9D2DA7F0A7E00125202758097
:10322800FF90F004E493F50AA3E493F50B90F007FC
:10323800E493F50CA3E493F50D850AA0850B80D2E1
:10324800DBC2DB7580FF00001257878F807590788E
:10325800D2B3C2B275907A75905AE4FFFE000000AE
:103268000000000FBF00010EEF64064E70EF75906E
:1032780058D2B2759078E50AB50C06E50B650D6075
:103288000A050BE50B70B2050A80AE7F067E0012B8
:10329800520275907CE4FEFF0000000000000FBFA2
:0932A80000010EEF64144E70EFFA
:0132B10022FA
:101C0B00E4F510F50FF50EF50D125A0A7F017E0063
:101C1B00125202C2B5D2D9D2DA7F0A7E0012520218
:101C2B007590FF90F004E493FBA3E493FA90F00714
:101C3B00E493F50AA3E493F98BA08A80D2DBC2DB91
:101C4B007580FF0000000000007590F80000C2B224
:101C5B00C2B3000000000000AF80000000000000D5
:101C6B00000000000000D2B3D2B2E4FCFDFEE51090
:101C7B002FF510EE350FF50FED350EF50EEC350D8E
:101C8B00F50DEBB50A04EA6960070AEA70AA0B8046
:101C9B00A77F067E0012520275907CAF10AE0FAD7F
:101CAB000EAC0D7810120A12AB07AF10AE0FAD0EC3
:101CBB00AC0D7808120A128F0BE510FFE48F0CAFF6
:101CCB0003FE1255A7125787AF0B7E001255A712B2
:091CDB005787AF0C7E000255A7EB
:103E5100750AAA125A0A7F0A7E00125202C2B5C21C
:103E6100D9D2DA7F0A7E001252027590DB0000007F
:103E71000000000000C2B2E4F50BF50C00000000E8
:103E81000000050CE50C7002050B6432450B70EC6B
:103E9100D2B27F067E00125202D2D97590FFE4F5AC
:103EA100A0F580D2DBC2DB7580FF7590F80000C2FF
:103EB100B2C2B3AF80000000000000D2B3D2B2EFB3
:103EC10060037F5522E4F50BF50C000000000000B3
:103ED100050CE50C7002050B6428450B70EC759020
:033EE100FF7FAAB6
:013EE40022BB
:1030B000750FAAE4F510F511125A0A7F017E00126D
:1030C0005202C2B5D2D9D2DA7F0A7E0012520275FC
:1030D00090FF7834E6F50B08E6F50C7837E6F50D49
:1030E00008E6F50E850BA0850C80D2DBC2DB75806F
:1030F000FF7590F80000C2B2C2B3000000000000EB
:1031000085800A000000000000D2B3D2B2AF0A7E70
:10311000001255A70511E51170020510B40029E54C
:1031200010B402241257878F0FE50A650F600D7FD8
:10313000557E001255A7150B150B80077FAA7E0040
:103140001255A7E4F510F511E50BB50D06E50C6574
:0D3150000E600A050CE50C708B050B8087E6
:01315D00224F
:1032B200125A0A7F017E00125202C2B57F047E00BA
:1032C200125202C2D9D2DA7F0A7E001252027580ED
:1032D200FF90F004E493FDA3E493FC90F007E493E1
:1032E200F50AA3E493F98DA08C80D2DBC2DB758052
:1032F200FF000075BF08EDFEEC7A002400FFEA3EF5
:103302008F82F583E0F58075BF02759078D2B3C2E3
:10331200B275907A75905AE4FFFE0000000000003A
:103322000FBF00010EEF64064E70EF759058D2B2D7
:10333200759078EDB50A04EC6960070CEC70A70D86
:1033420080A4E4FEFF0000000000000FBF00010E99
:06335200EF64144E70EF61
:013358002252
:10492900750CAA125A0A7F017E00125202C2B5D230
:10493900D9D2DA7F0A7E001252027590FF90F004F4
:10494900E493FDA3E493FC90F007E493F50AA3E450
:1049590093F50B8DA08C80D2DBC2DB7580FF75903F
:10496900F80000C2B2C2B3A980000000000000D262
:10497900B3D2B275BF08EDFEEC7A002400FFEA3E1F
:104989008F82F583E075BF026960037F5522EDB51B
:104999000A07ECB50B037FAA220CEC70B60D80B3A5
:1012F000E4F513F512F511F510F514F515125A0A67
:10130000C2B57834E6F50A08E6F50B7837E6F50C51
:1013100008E6F50D75F65575F6AA75F65575BF0C08
:10132000E4F5F475F7A275F7A205F405F40515E5E3
:1013300015700205146480451470E8850AF4850B65
:10134000F51257878FF675F7A0E50AFE7C00E425B5
:101350000BFFEC3E8F82F583E0FFE4FDFEE5132FEB
:10136000F513EE3512F512ED3511F511EC3510F5DA
:1013700010E50AB50C06E50B650D600A050BE50BDB
:1013800070B9050A80B575BF02AF13AE12AD11ACCE
:10139000107810120A12AB07AF13AE12AD11AC10D9
:1013A0007808120A128F0EE513FFE48F0FAF03FEC9
:1013B0001255A7125787AF0E7E001255A7125787F6
:1013C000783AA6077B007A007930751B0BE4FD7F25
:0B13D000F01254C4AF0F7E000255A7BE
:1007FC007830E6146052146066146077147003024B
:10080C0008941470030208AB1470030208C024F59A
:10081C0070030208C9241160030209491259038F9D
:10082C0008E508B4AA0F1251937F1E7E00125202E3
:10083C0012519380347F1E7E001252027F557E002F
:10084C001255A7C2B40259B7124ECB8F087E0012B4
:10085C0055A7D2B5E508B4AA030209440209491206
:10086C003A2D7F017E001252027FAA7E001255A7FC
:10087C000209421226971257878F08D2B5E508B4A1
:10088C00AA03020944020949124A298F087E001260
:10089C0055A7D2B5E508B4AA0302094402094912C6
:1008AC0013DB1257878F08D2B5E508B4AA030209E7
:1008BC0044020949122DE5C2B6D2B5807D90F00AEA
:1008CC00E493F50930E0241259038F08E50864AA73
:1008DC00600AD2B5C2B41259B702596F1251937F44
:1008EC001E7E00125202125193D2B5E50930E11866
:1008FC00124ECB8F08E50864AA60028035C2B67F21
:10090C001E7E00125202D2B6E50930E20312353FC8
:10091C00E50930E30D12471A8F08E50864AA600256
:10092C008010E50930E40F124A298F08E50864AA03
:10093C006004D2B58007D2B5C2B6025A49C2B4120D
:02094C0059A0B0
:01094E002286
:10519300125A0A7F017E00125202C2B5C2D9D2DA74
:1051A3007F0A7E0012520275905E0000000000002C
:1051B300000000000000C2B2000000000000000078
:1051C3000000000075905F7FE87E03125202D2B2A6
:1051D300E4FFFE0000000000000FBF00010EEF64BB
:1051E300144E70EFD2D97590FF7F017E00025202F8
:104ECB00125A0A7F017E00125202C2B5D2D9D2DA2F
:104EDB007F0A7E001252027590FF90F004E493FF5C
:104EEB00A3E493FE90F007E493FDA3E493FC8FA05F
:104EFB008E80D2DBC2DB7580FFC2B20000C2B30072
:104F0B000000000000AB80000000000000D2B300E6
:104F1B0000D2B2EBF460037F5522EFB50507EEB577
:0C4F2B0004037FAA220EEE70C50F80C2A6
:103A2D00125A0A7F017E00125202C2B57F047E0037
:103A3D00125202C2D9D2DA7F0A7E0012520275806A
:103A4D00FF90F004E493F50AA3E493F50B90F007CF
:103A5D00E493F50CA3E493F50D850AA0850B80D2B4
:103A6D00DBC2DB7580FF00001257878F8075905782
:103A7D000000C2B2000075905FE4FFFE0000000080
:103A8D0000000FBF00010EEF64044E70EFD2B2E5DF
:103A9D000AB50C06E50B650D600A050BE50B70B953
:103AAD00050A80B5E4FEFF0000000000000FBF0016
:083ABD00010EEF641E4E70EFD4
:013AC50022DE
:10269700E4F510F50FF50EF50D125A0A7F017E00CD
:1026A700125202C2B5D2D9D2DA7F0A7E0012520282
:1026B7007590FF90F004E493FBA3E493FA90F0077E
:1026C700E493F50AA3E493F98BA08A80D2DBC2DBFB
:1026D7007580FFC2B20000C2B3000000000000AF67
:1026E70080000000000000D2B30000D2B2E4FCFD7D
:1026F700FEE5102FF510EE350FF50FED350EF50E43
:10270700EC350DF50DEBB50A04EA6960070AEA70C6
:10271700B70B80B4AF10AE0FAD0EAC0D7810120A28
:1027270012AB07AF10AE0FAD0EAC0D7808120A1240
:102737008F0BE510FFE48F0CAF03FE1255A712575E
:1027470087AF0B7E001255A7125787AF0C7E00028A
:0227570055A784
:104A2900125A0A7F0A7E00125202C2B5C2D9D2DADC
:104A39007F0A7E001252027590CF0000000000002C
:104A4900C2B20000000000007590DFE4FFFE000024
:104A5900000000000FBF00010EEF64324E70EFD26C
:104A6900B2000000000000D2D97590FFE4F5A0F56E
:104A790080D2DBC2DB7580FFC2B20000C2B3000086
:104A890000000000AF80000000000000D2B3000069
:0D4A9900D2B2EF60037F55227590FF7FAA17
:014AA60022ED
:102DE500E4F50FF510125A0A7F017E00125202C255
:102DF500B5D2D9D2DA7F0A7E001252027590FF78D9
:102E050034E6F50B08E6F50C7837E6F50D08E6F53A
:102E15000E850BA0850C80D2DBC2DB7580FFC2B2AC
:102E25000000C2B300000000000085800A00000019
:102E3500000000D2B30000D2B2AF0A7E001255A73F
:102E45000000000000000000000000000510E51073
:102E55007002050FB40026E50FB40221125787E56D
:102E65000A6F600D7F557E001255A7150B150B8057
:102E7500077FAA7E001255A7E4F50FF510E50BB5FF
:102E85000D06E50C650E600B050CE50C7083050B56
:032E9500022E16F4
:012E98002217
:1013DB00E4F513F512F511F510F514F515125A0A7B
:1013EB00C2B57834E6F50A08E6F50B7837E6F50C66
:1013FB0008E6F50D75F65575F6AA75F65575BF0C1D
:10140B00E4F5F475F7A275F7A205F405F40515E5F7
:10141B0015700205146480451470E8850AF4850B79
:10142B00F51257878FF675F7A0E50AFE7C00E425C9
:10143B000BFFEC3E8F82F583E0FFE4FDFEE5132FFF
:10144B00F513EE3512F512ED3511F511EC3510F5EE
:10145B0010E50AB50C06E50B650D600A050BE50BEF
:10146B0070B9050A80B575BF02AF13AE12AD11ACE2
:10147B00107810120A12AB07AF13AE12AD11AC10ED
:10148B007808120A128F0EE513FFE48F0FAF03FEDD
:10149B001255A7125787AF0E7E001255A71257870A
:1014AB00783AA6077B007A007930751B0BE4FD7F39
:0B14BB00F01254C4AF0F7E000255A7D2
:10353F00125A0A7F017E00125202C2B57F047E002A
:10354F00125202C2D9D2DA7F0A7E0012520275805D
:10355F00FF90F004E493FDA3E493FC90F007E49351
:10356F00F50AA3E493F98DA08C80D2DBC2DB7580C2
:10357F00FF000075BF08EDFEEC7A002400FFEA3E65
:10358F008F82F583E0F58075BF027590570000C2FA
:10359F00B2000075905FE4FFFE0000000000000F16
:1035AF00BF00010EEF64054E70EFD2B2EDB50A0405
:1035BF00EC6960070CEC70AE0D80ABE4FEFF000011
:0F35CF00000000000FBF00010EEF64284E70EFE8
:0135DE0022CA
:10471A00750CAA125A0A7F017E00125202C2B5D241
:10472A00D9D2DA7F0A7E001252027590FF90F00405
:10473A00E493FDA3E493FC90F007E493F50AA3E461
:10474A0093F50B8DA08C80D2DBC2DB7580FFC2B2E1
:10475A000000C2B3000000000000A98000000000B1
:10476A000000D2B30000D2B275BF08EDFEEC7A00A9
:10477A002400FFEA3E8F82F583E075BF0269600379
:10478A007F5522EDB50A07ECB50B037FAA220CEC84
:05479A0070B10D80AEBE
:1006A0007830E6120A2506C50006FB01071202078C
:1006B0003E03075204076805077C06078507079570
:1006C00011000007F6C29612555DC2967F057E00A6
:1006D000125202E4FF125070C2967F057E00125241
:1006E000021255118F08E50860028044123AC67F55
:1006F0001E7E00125202123AC6803F1245008F0839
:100700007E001255A7D2B5E508B4AA0302079102EC
:1007100007F6122BBF12555D12506A1255118F0841
:100720007F017E0012520290F002E4936508600A95
:100730007F557E001255A70207EB7FAA804C121B43
:100740002B1257878F08D2B5E508B4AA028042025F
:1007500007F61243EC8F087E001255A7D2B5E508C4
:10076000B4AA02802C0207F61214C61257878F080B
:10077000D2B5E508B4AA0280180207F612210BC20E
:10078000B6D2B5806E1255118F087E001255A7D2D1
:10079000B5C2B6805E90F00AE493F50930E00D1220
:1007A0003AC67F1E7E00125202123AC6E50930E1B7
:1007B0000D1245008F08E50864AA6002802DE50946
:1007C00030E20612275912506AE50930E30D12256E
:1007D000088F08E50864AA60028010E50930E40F7C
:1007E0001243EC8F08E50864AA6004D2B58007D2F2
:0B07F000B5C2B6025A49C2B41259A0AB
:0107FB0022DB
:103AC600125A0A7F017E00125202C2B5D2B37F019A
:103AD6007E001252027590C3D2DBC2DBD2B275A051
:103AE600FF7580FFD2D9C2DA000000000000759091
:103AF60043E4FFFE0000000000000FBF00010EEFD0
:103B0600641E4E70EF7590C37F4C7E04125202D233
:103B1600D9D2DA7F1E7E001252027590C3D2DBC262
:103B2600DBD2B275A0FF7580FFD2D9C2DA000000E1
:103B3600000000759043E4FEFF0000000000000F47
:103B4600BF00010EEF641E4E70EF7590C37F4C7E72
:083B560004125202D2D9D2DAA6
:013B5E002244
:10450000125A0A7F017E00125202C2B57F0A7E0053
:10451000125202D2D9C2DA7F017E0012520290F00A
:1045200003E493FFA3E493FEA3E493FDA3E493F5D4
:104530000AA3E493F9A3E493FBEF1392B28EA08D48
:1045400080D2DBC2DB7580FF7590C0C2DA0000004C
:10455000000000C2B3AC80000000000000D2B30035
:104560000000000000D2DAECF460037F5522EFB5C2
:104570000A0BEEB50107EDB503037FAA220DED701E
:08458000B80EEE70B40F80B11B
:102BBF00125A0A7F017E00125202C2B5D2D9C2DA6E
:102BCF007F0A7E001252027580FF90F003E493F5A6
:102BDF000AA3E493F50BA3E493F50CA3E493F50D8B
:102BEF00A3E493F50EA3E493F50FE50A1392B285D0
:102BFF000BA0850C80D2DBC2DB7580FF0000125763
:102C0F00878F807590C00000C2DA000000000000BE
:102C1F0000000000000075904000007590C0E4FFB8
:102C2F00FE0000000000000FBF00010EEF64034E16
:102C3F0070EFD2DAE50AB50D0BE50BB50E06E50C14
:102C4F00650F6010050CE50C70A0050BE50B709A75
:102C5F00050A8096E4FEFF0000000000000FBF0091
:082C6F00010EEF64284E70EF26
:012C7700223A
:101B2B00E4F512F511F510F50F125A0A7F017E003C
:101B3B00125202C2B57F0A7E00125202D2D9C2DA09
:101B4B007F017E0012520290F003E493F9A3E49319
:101B5B00FBA3E493FAA3E493F50AA3E493F50BA395
:101B6B00E493F50CE91392B28BA08A80D2DBC2DB33
:101B7B007580FF7590C0C2DA000000000000C2B390
:101B8B00AF80000000000000D2B300000000000096
:101B9B00D2DAE4FCFDFEE5122FF512EE3511F5114C
:101BAB00ED3510F510EC350FF50FE9B50A09EBB56E
:101BBB000B05EA650C600B0AEA70A90BEB70A50923
:101BCB0080A2AF12AE11AD10AC0F7810120A12AB8F
:101BDB0007AF12AE11AD10AC0F7808120A128F0DB1
:101BEB00E512FFE48F0EAF03FE1255A7125787AF16
:101BFB000D7E001255A7125787AF0E7E000255A718
:1043EC00750AAA125A0A7F017E00125202C2B5D275
:1043FC00D9C2DA7F0A7E001252027590C1C2DAE489
:10440C00FFFE0000000000000FBF00010EEF64462D
:10441C004E70EF75904100007590C1E4FEFF0000F6
:10442C00000000000FBF00010EEF64324E70EFD29F
:10443C00DA7590FFC2B2E4F5A0F580D2DBC2DB7571
:10444C0080FF7590C0C2DA000000000000C2B3AF5C
:10445C0080000000000000D2B3000000000000D279
:09446C00DAEF60037F55227FAAFC
:014475002224
:10210B00E4F511F512125A0A7F017E00125202C237
:10211B00B57F0A7E00125202D2D9C2DA7F017E004D
:10212B001252027833E6F50B08E6F50C08E6F50DCE
:10213B0008E6F50E08E6F50F08E6F510E50B24FFAB
:10214B0092B2850CA0850D80D2DBC2DB7580FF754A
:10215B0090C0C2DA000000000000C2B385800A0004
:10216B000000000000D2B3000000000000D2DAAF84
:10217B000A7E001255A70512E51270020511B40074
:10218B0026E511B40221125787E50A6F600D7F55C2
:10219B007E001255A7150C150C80077FAA7E001226
:1021AB0055A7E4F511F512E50BB50E0BE50CB50FC4
:1021BB0006E50D65106017050DE50D60030221475F
:0E21CB00050CE50C6003022147050B022147BD
:0121D90022E3
:06506A0090F002E493FF48
:025070008F0AA5
:10507200E50A25E0F50A125A0A7F0A7E0012520258
:10508200C2B5C2B275A0010000850A800000D2DB61
:10509200C2DB7590ECD2B3D2D9C2DA0000000000B4
:1050A2000000000000000075906C0000000000008D
:1050B2007590ECE4FFFE0000000000000FBF00014D
:0B50C2000EEF642E4E70EFD2D9D2DA50
:0150CD0022C0
:10555D00125A0A7F0A7E00125202C2B57590E0D22D
:10556D00B3C2B275A001E4F580000000000000D2C6
:10557D00D9C2DA000000000000D2DBC2DB0000005F
:10558D000000007590600000000000007590E07F45
:0A559D000AFE125202D2D9D2DA221D
:10551100125A0A7F017E00125202C2B5D2DBC2DBEF
:105521007590C1D2B275A0FF000000000000D2D971
:10553100C2DA000000000000000000000000C2B359
:10554100000000000000AF80D2B3000000000000A6
:0B555100D2D9D2DA000000007590C330
:01555C00222C
:10275900125A0A7F017E00125202C2B5D2D9C2DAD8
:102769007F0A7E001252027580FF90F003E493F90C
:10277900A3E493FDA3E493FBA3E493F50AA3E493F1
:10278900F50BA3E493F50CE924FF92B28DA08B809D
:10279900D2DBC2DB7580FF000075BF08EDFEEB756B
:1027A90083002400FFE5833E8F82F583E0F5807581
:1027B900BF027590C00000C2DA00000000000000EE
:1027C900000000000075904000007590C0E4FFFE15
:1027D9000000000000000FBF00010EEF64034E70FF
:1027E900EFE9B50A09EDB50B05EB650C600B0BEBD1
:1027F90070950DED709109808EE4FEFF00000000D8
:0D28090000000FBF00010EEF64284E70EFBD
:01281600229F
:10250800125A0A7F017E00125202C2B57F0A7E006B
:10251800125202D2D9C2DA7F017E0012520290F022
:1025280003E493F50BA3E493F50CA3E493F50DA34F
:10253800E493F50EA3E493F50FA3E493F510E50BEC
:1025480024FF92B2850CA0850D80D2DBC2DB75809A
:10255800FF7590C0000000000000C2B385800A002B
:102568000000000000D2B300000000000075BF08A2
:10257800AF0BE4FCFDFEFBFA7901F81209B2AD07D6
:10258800AC06E50CFEE42DFFEE3CFE7C00EF250DCD
:10259800FFEC3E8F82F583E075BF02650A60037F1A
:1025A8005522E50BB50E0DE50CB50F08E50DB51078
:1025B800037FAA22050DE50D7084050CE50C600368
:0825C800022546050B02254621
:1014C600E4F513F512F511F510F514F515125A0A8F
:1014D600C2B57834E6F50A08E6F50B7837E6F50C7A
:1014E60008E6F50D75F65575F6AA75F65575BF0C31
:1014F600E4F5F475F7A275F7A205F405F40515E50C
:1015060015700205146480451470E8125787850A21
:10151600F4850BF58FF675F7A0E50AFE7C00E42549
:101526000BFFEC3E8F82F583E0FFE4FDFEE5132F13
:10153600F513EE3512F512ED3511F511EC3510F502
:1015460010E50AB50C06E50B650D600A050BE50B03
:1015560070B9050A80B575BF02AF13AE12AD11ACF6
:10156600107810120A12AB07AF13AE12AD11AC1001
:101576007808120A128F0EE513FFE48F0FAF03FEF1
:101586001255A7125787AF0E7E001255A71257871E
:10159600783AA6077B007A007930751B0BE4FD7F4D
:0B15A600F01254C4AF0F7E000255A7E6
:100003007830E6120A25002800005C01007802001F
:10001300AF0300C30400D90500ED0600F60701078E
:1000230011000001B51255EFE4FF1251381256C406
:100033008F08E508600BD2B5C2B41259A07F558072
:10004300661258767F1E7E00125202125876D2B57F
:10005300C2B6125A497FAA804E1248238F08D2B5DE
:10006300E508B4AA07C2B6125A498005C2B41259A8
:10007300A0AF0880321237BE1255EF12513212561A
:10008300C48F087F017E0012520290F002E4936550
:1000930008600BD2B5C2B41259A07F558009D2B5FE
:1000A300C2B6125A497FAA7E000255A7121DBC127E
:1000B30057878F08D2B5E508B4AA0280420201B57A
:1000C3001242D48F087E001255A7D2B5E508B4AA10
:1000D30002802C0201B51210211257878F08D2B566
:1000E300E508B4AA0280180201B512298EC2B6D25D
:1000F300B5800E1256C48F087E001255A7D2B5C222
:10010300B6025A4990F00AE493F50930E0281255F3
:10011300EFE4FF1251381256C48F08E5086003025A
:1001230001A71258767F1E7E00125202125876D211
:10013300B5C2B6125A49E50930E1141248238F08B3
:10014300E50864AA6002805CD2B5C2B6125A49E5DA
:100153000930E2271233591255EF1251321256C4A5
:100163008F087F017E0012520290F002E49365082B
:1001730060028030D2B5C2B6125A49E50930E314A1
:10018300123EE58F08E50864AA60028017D2B5C263
:10019300B6125A49E50930E4161242D48F08E5082D
:1001A30064AA6004D2B5800AD2B5C2B6125A490213
:0701B300596FC2B41259A0FC
:0101BA002222
:10587600125A0A7F017E00125202C2B5D2D9C2DA8A
:105886007590F0C2B2000075907000007590F0003F
:0F589600007FB07E04125202D2B2D2D9D2DA22EF
:10482300125A0A7F017E00125202C2B57F0A7E002D
:10483300125202D2D9C2DA7F017E0012520290F0E4
:1048430004E493FFA3E493FE90F007E493FDA3E451
:1048530093FC8FA08E80D2DBC2DB7580FF7590C086
:10486300000000000000C2B2000000000000C2B35C
:10487300000000000000AB80D2B300000000000085
:10488300D2B2EBF46007D2D9D2DA7F5522EFB50565
:104893000BEEB50407D2D9D2DA7FAA220EEE70B29C
:0348A3000F80AFD4
:1037BE00125A0A7F017E00125202C2B5D2D9C2DA63
:1037CE007F0A7E001252027580FF90F004E493F59A
:1037DE000AA3E493F50B90F007E493F50CA3E4939E
:1037EE00F50D850AA0850B80D2DBC2DB7580FF004C
:1037FE00001257878F807590C0D2B3C2B200007589
:10380E00904000007590C0E4FFFE00000000000034
:10381E000FBF00010EEF64054E70EFD2B2E50AB590
:10382E000C0BE50BB50D06D2D9D2DA800A050BE5E5
:10383E000B70AF050A80ABE4FEFF00000000000035
:0B384E000FBF00010EEF64284E70EF6A
:01385900224C
:101DBC00E4F511F510F50FF50E125A0A7F017E00AD
:101DCC00125202C2B57F0A7E00125202D2D9C2DA76
:101DDC007F017E0012520290F004E493FBA3E49383
:101DEC00FA90F007E493F50AA3E493F98BA08A80A8
:101DFC00D2DBC2DB7580FF7590C0000000000000D4
:101E0C00C2B20000C2B3000000000000AF80D2B329
:101E1C000000D2B2E4FCFDFEE5112FF511EE3510F9
:101E2C00F510ED350FF50FEC350EF50EEBB50A0A86
:101E3C00EAB50106D2D9D2DA80070AEA70AE0B8075
:101E4C00ABAF11AE10AD0FAC0E7810120A128F0B97
:101E5C00AF11AE10AD0FAC0E7808120A128F0CE554
:101E6C0011FFE48F0D7F0AFE125202AF0B7E00129F
:101E7C0055A7125787AF0C7E001255A7125787AF84
:061E8C000D7E000255A7C7
:1042D400750AAA125A0A7F017E00125202C2B5D28E
:1042E400D9C2DA7F017E001252027590D00000C25A
:1042F400B275905000007590D0E4FFFE00000000FD
:1043040000000FBF00010EEF64324E70EFD2B275A1
:1043140090FFE4FEFF0000000000000FBF00010E4C
:10432400EF64144E70EFE4F5A0F580D2DBC2DB75C8
:1043340080FF7590C0000000000000C2B20000C2FF
:10434400B3000000000000AF80D2B30000D2B2D2AC
:0B435400D9D2DAEF60037F55227FAA68
:01435F00223B
:10298E00750FAAE4F510F511125A0A7F017E001296
:10299E005202C2B57F0A7E00125202D2D9C2DA7F2B
:1029AE00017E001252027834E6F50B08E6F50C783B
:1029BE0037E6F50D08E6F50E850BA0850C80D2DB0B
:1029CE00C2DB7580FF7590C0000000000000C2B22F
:1029DE000000C2B300000000000085800AD2B300E0
:1029EE0000D2B2AF0A7E001255A70511E511700292
:1029FE000510B4002FE510B4022A1257878F0FE589
:102A0E000A650F600D7F557E001255A7150B150B2D
:102A1E0080077FAA7E001255A7E4F510F5117F14EA
:102A2E00FE125202E50BB50D06E50C650E600B05A8
:0A2A3E000CE50C7083050B0229C69D
:012A4800226B
:1055EF00125A0A7F017E00125202C2B5D2D9C2DA14
:1055FF007F017E001252027590C8000075A0010055
:10560F0000E4F5800000D2DBC2DB0000C2B2000074
:10561F0075904800007590C800007F0AFE12520274
:07562F00D2B2D2D9D2DA2277
:0651320090F002E493FF7F
:025138008F0ADC
:10513A00125A0A7F017E00125202C2B5E50A25E020
:10514A00F50AD2D9C2DA7F017E0012520275A00195
:10515A000000850A800000D2DBC2DB7590CBC2B2A8
:10516A00000075904B00007590CB0000E4FFFE0034
:10517A0000000000000FBF00010EEF64294E70EF1F
:08518A000000D2B2D2D9D2DA42
:0151920022FA
:1056C400125A0A7F017E00125202C2B5D2D9C2DA3E
:1056D4007F017E00125202E4F5A0F580D2DBC2DB2A
:1056E4007580FF7590D0C2B2C2B300000000000004
:1056F400759050AF807590D0D2B3D2B2D2D9D2DAED
:015704002282
:10335900125A0A7F017E00125202C2B5D2D9C2DACC
:103369007F0A7E001252027580FF90F004E493FDFB
:10337900A3E493FC90F007E493F50AA3E493F98D91
:10338900A08C80D2DBC2DB7580FF000075BF08ED21
:10339900FEEC7A002400FFEA3E8F82F583E0F58097
:1033A90075BF027590C0D2B3C2B2000075904000DB
:1033B900007590C0E4FFFE0000000000000FBF0090
:1033C900010EEF64054E70EFD2B2EDB50A0AECB505
:1033D9000106D2D9D2DA80070CEC70A30D80A0E4E3
:1033E900FEFF0000000000000FBF00010EEF64287F
:0333F9004E70EF24
:0133FC0022AE
:103EE500750CAA125A0A7F017E00125202C2B57FD2
:103EF5000A7E00125202D2D9C2DA7F017E00125226
:103F05000290F004E493FDA3E493FC90F007E4939E
:103F1500F50AA3E493F50B8DA08C80D2DBC2DB758B
:103F250080FF7590C0000000000000C2B20000C212
:103F3500B3000000000000A980D2B30000D2B27522
:103F4500BF08EDFEEC7A002400FFEA3E8F82F58380
:103F5500E075BF02696007D2D9D2DA7F5522EDB587
:103F65000A0BECB50B07D2D9D2DA7FAA220CEC707A
:043F7500A60D80A372
:10102100E4F513F512F511F510F514F515125A0A38
:10103100C2B57834E6F50A08E6F50B7837E6F50C23
:1010410008E6F50D75F65575F6AA75F65575BF0CDA
:10105100E4F5F475F7A275F7A205F405F40515E5B5
:1010610015700205146480451470E8850AF4850B37
:10107100F51257878FF675F7A0E50AFE7C00E42587
:101081000BFFEC3E8F82F583E0FFE4FDFEE5132FBD
:10109100F513EE3512F512ED3511F511EC3510F5AC
:1010A10010E50AB50C06E50B650D600A050BE50BAD
:1010B10070B9050A80B575BF027F0A7E001252021F
:1010C100AF13AE12AD11AC107810120A12AB07AF0C
:1010D10013AE12AD11AC107808120A128F0EE5137F
:1010E100FFE48F0FAF03FE1255A7125787AF0E7E95
:1010F100001255A7125787783AA6077B007A007924
:1011010030751B0BE4FD7FF01254C4AF0F7E00025B
:0211110055A7E0
:100373007830E614607A14700302040814700302E0
:10038300041D147003020430147003020445147036
:100393000302045D24F57003020467241160030261
:1003A300051D12592E1259038F08E50864AA702DF2
:1003B3001258407F1E7E001252021258407F1E7E4A
:1003C300001252021258407F1E7E0012520212582F
:1003D300407F1E7E0012520212584080327F1E7EE2
:1003E300001252027F557E001255A7C2B40259B7BC
:1003F30012460F8F087E001255A7D2B5E508B4AA9E
:100403000280268050122E997F017E001252027FB5
:10041300AA7E001255A7D2B58037121CE412578763
:100423008F08D2B5E508B4AA028026802812412D90
:100433008F087E001255A7D2B5E508B4AA02801131
:1004430080131215B11257878F08D2B5E508B4AAE5
:1004530004C2B6800CC2B40259A012203AC2B6D26A
:10046300B5025A4990F00AE493F50930E045125970
:100473002E1259038F08E50864AA600AD2B5C2B4E4
:100483001259B70205221258407F1E7E00125202F3
:100493001258407F1E7E001252021258407F1E7E69
:1004A300001252021258407F1E7E0012520212584E
:1004B30040D2B5E50930E11F12460F8F08E5086405
:1004C300AA6009D2B5C2B41259A08053C2B67F1E26
:1004D3007E00125202D2B6E50930E203122A49E540
:1004E3000930E31412385A8F08E50864AA6009D268
:1004F300B5C2B41259A08027E50930E41412412D86
:100503008F08E50864AA6009D2B5C2B41259A08065
:100513000ED2B5C2B6125A498005C2B41259A012FE
:02052300596F0E
:0105250022B3
:10584000125A0A7F017E00125202C2B512592EC2AC
:10585000D97F0A7E0012520275907B758083759005
:10586000FB000075907B7590737FF47E01125202ED
:0658700075907BD2D922E5
:10460F00750AAA12592E7F017E00125202C2B5C23C
:10461F00D97F0A7E001252027580FF90F004E49356
:10462F00FFA3E493FE90F007E493FDA3E493FC75DE
:10463F0090788F807590F800007590787580FF7571
:10464F0090798E807590F9000075907975907BE464
:10465F00F5807590FB000075907B7580FF759073EA
:10466F000000AB8075907B000000000000EBF46051
:10467F00037F5522EFB50507EEB504037FAA220E7F
:06468F00EE70AC0F80A9E3
:102E990012592E7F017E00125202C2B5C2D97F0A91
:102EA9007E001252027580FF90F004E493F50AA3A4
:102EB900E493F50B90F007E493F50CA3E493F50D77
:102EC90012578775907C850A807590FC0000759073
:102ED9007C7580FF75907D850B807590FD00007570
:102EE900907D75907E8F807590FE000075907E753F
:102EF900907F7580237590FF000075907F7580FF26
:102F0900759077E4FFFE0000000000000FBF00018C
:102F19000EEF64064E70EF75907CE50AB50C06E578
:102F29000B650D600A050BE50B7095050A8091E4A8
:102F3900FEFF0000000000000FBF00010EEF641447
:032F49004E70EFD8
:012F4C002262
:101CE400E4F510F50FF50EF50D12592E7F017E0067
:101CF400125202C2B5C2D97F0A7E00125202758006
:101D0400FF90F004E493FBA3E493FA90F007E493C8
:101D1400F50AA3E493F97590788B807590F8000028
:101D24007590787580FF7590798A807590F90000B8
:101D340075907975907BE4F5807590FB0000759043
:101D44007B7580FF7590730000AF8075907B0000F9
:101D540000000000FCFDFEE5102FF510EE350FF538
:101D64000FED350EF50EEC350DF50DEBB50A04EA65
:101D74006960070AEA709F0B809CAF10AE0FAD0E2E
:101D8400AC0D7810120A12AB07AF10AE0FAD0EAC4B
:101D94000D7808120A128F0BE510FFE48F0CAF03C5
:101DA400FE1255A7125787AF0B7E001255A7125784
:081DB40087AF0C7E000255A769
:10412D00750AAA12592E7F017E00125202C2B5C223
:10413D00D97F0A7E001252027580FF75907B7580C3
:10414D00137590FB000075907B7580FF7590737FE4
:10415D00017E0012520275907BD2D9C2D97F017EA9
:10416D0000125202759078E4F5807590F800007594
:10417D0090787580FF759079F5807590F9000075D0
:10418D0090797580FF75907BF5807590FB000075BB
:10419D00907B7580FF7590730000AF8075907B00EC
:0D41AD000000000000EF70037FAA227F5584
:0141BA0022E2
:10203A00750FAAC200E4F510F51112592E7F017E20
:10204A0000125202C2B5C2D97F0A7E00125202752C
:10205A0080FF90F004E493F50BA3E493F50C90F061
:10206A0007E493F50DA3E493F50E759078850B803C
:10207A007590F800007590787580FF759079850CD9
:10208A00807590F9000075907975907BE4F58075FC
:10209A0090FB000075907B7580FF7590730000853A
:1020AA00800A75907B000000000000AF0AFE1255FE
:1020BA00A70511E51170020510B4002BE510B40252
:1020CA00261257878F0FE50A650F600F7F557E002E
:1020DA001255A7150B150BC20080077FAA7E0012A6
:1020EA0055A7E4F510F511E50BB50D06E50C650EDF
:1020FA00600E050CE50C6003022074050B022074C7
:01210A0022B2
:102A490012592E7F017E00125202C2B5C2D97F0AE5
:102A59007E001252027580FF90F004E493FDA3E416
:102A690093FC90F007E493F50AA3E493F975BF0882
:102A7900EDFEEC7A002400FFEA3E8F82F583E075D3
:102A8900BF0275907C8D807590FC000075907C75F7
:102A990080FF75907D8C807590FD000075907D7527
:102AA900907EF5807590FE000075907E75907F751B
:102AB90080237590FF000075907F7580FF75907772
:102AC900E4FFFE0000000000000FBF00010EEF64EC
:102AD900064E70EF75907CEDB50A04EC6960070C41
:102AE900EC708A0D8087E4FEFF0000000000000FF3
:0A2AF900BF00010EEF64144E70EFF1
:012B030022AF
:10385A00750CAA12592E7F017E00125202C2B5C2FD
:10386A00D97F0A7E001252027580FF90F004E49319
:10387A00FDA3E493FC90F007E493F50AA3E493F51F
:10388A000B7590788D807590F8000075907875802A
:10389A00FF7590798C807590F90000759079759014
:1038AA007BE4F5807590FB000075907B7580FF7551
:1038BA0090730000A98075907B00000000000075DD
:1038CA00BF08EDFEEC7A002400FFEA3E8F82F58302
:1038DA00E075BF02696002890CEDB50A05EC650B5B
:0B38EA0060070CEC709B0D8098AF0C89
:0138F50022B0
:1015B100E4F513F512F511F510F514F515125A0AA3
:1015C100C2B57834E6F50A08E6F50B7837E6F50C8E
:1015D10008E6F50D75F65575F6AA75F65575BF0C45
:1015E100E4F5F475F7A275F7A205F405F40515E520
:1015F10015700205146480451470E8125787850A36
:10160100F4850BF58FF675F7A0E50AFE7C00E4255D
:101611000BFFEC3E8F82F583E0FFE4FDFEE5132F27
:10162100F513EE3512F512ED3511F511EC3510F516
:1016310010E50AB50C06E50B650D600A050BE50B17
:1016410070B9050A80B575BF02AF13AE12AD11AC0A
:10165100107810120A12AB07AF13AE12AD11AC1015
:101661007808120A128F0EE513FFE48F0FAF03FE05
:101671001255A7125787AF0E7E001255A712578732
:10168100783AA6077B007A007930751B0BE4FD7F61
:0B169100F01254C4AF0F7E000255A7FA
:10592E00E4FFFED2B4D2B5D2B67590FFF580D2DACE
:10593E00D2D9C2970FBF00010ED297EF64644E709A
:01594E00F167
:01594F002235
:100BDE007830E6120A250C03000C12010C28020CC8
:100BEE0039030C4D040C63050C77060C80070C9032
:100BFE001100000CFC123F797F1E7E001252021271
:100C0E003F7980231245888F4A7E001255A7D2B5B0
:100C1E00E54AB4AA028067020CFC123B5F1248A69A
:100C2E007F017E001252027FAA804C121E92125732
:100C3E00878F4AD2B5E54AB4AA028042020CFC1252
:100C4E0041BB8F4A7E001255A7D2B5E54AB4AA021F
:100C5E00802C020CFC12169C1257878F4AD2B5E5D7
:100C6E004AB4AA028018020CFC122F4DC2B6D2B59D
:100C7E0080791258058F4A7E001255A7D2B5C2B69A
:100C8E00806990F00AE493F54B30E00D123F797FC6
:100C9E001E7E00125202123F79E54B30E1181245CA
:100CAE00888F4AE54A64AA60028038C2B67F1E7EEB
:100CBE0000125202D2B6E54B30E2061238F6124856
:100CCE00A6E54B30E30D1244768F4AE54A64AA60DE
:100CDE00028010E54B30E40F1241BB8F4AE54A64A7
:100CEE00AA6004D2B58007D2B5C2B6025A49C2B4C0
:030CFE001259A0E8
:010D010022CF
:103F7900125A0A7F017E00125202C2B5C2D97F01CC
:103F89007E001252027590C8000075A0010000E47D
:103F9900F5800000D2DBC2DB0000C2B200007590E0
:103FA9004800007590C800007F0AFE125202D2B282
:103FB90075A0010000E4F5800000D2DBC2DB75903A
:103FC900CBC2B2000075904B00007590EC0000FF69
:103FD900FE0000000000000FBF00010EEF64294E33
:103FE90070EF0000D2B27590F0C2B2000075907007
:103FF90000007590F000007FDC7E05125202D2B2FB
:02400900C2D91A
:01400B002292
:10458800754CAA125A0A7F017E00125202C2B57FE8
:104598000A7E00125202C2D97F017E001252029096
:1045A800F004E493FFA3E493FE90F007E493FDA3E3
:1045B800E493FC8FA08E80D2DBC2DB7580FF759000
:1045C800C0000000000000C2B2000000000000C2ED
:1045D800B300000000000000000000000000000020
:1045E800000000AB80D2B3000000000000D2B2EBA4
:1045F800F460028B4CEFB50504EE6C60070EEE70AC
:06460800B20F80AFAF4CC1
:01460E002289
:103B5F00125A0A7F0A7E00125202C2B5C2D97F0AD8
:103B6F007E001252027580FF90F004E493F51CA3BF
:103B7F00E493F51D90F007E493F51EA3E493F51F6E
:103B8F00125787851CA0851D80D2DBC2DB7580FF95
:103B9F000000000000008F807590C0D2B3C2B20049
:103BAF000075904000007590C0E4FFFE000000001B
:103BBF0000000FBF00010EEF64064E70EFD2B2E5AA
:103BCF001CB51E06E51D651F600A051DE51D70B0BD
:103BDF00051C80ACE4FEFF0000000000000FBF00DA
:083BEF00010EEF64284E70EF97
:013BF70022AB
:101E9200E4F549F548F547F546125A0A7F017E00F6
:101EA200125202C2B57F0A7E00125202C2D97F01CB
:101EB2007E0012520290F004E493FBA3E493FA90A2
:101EC200F007E493F543A3E493F98BA08A80D2DB75
:101ED200C2DB7580FF7590C0000000000000C2B236
:101EE200000000000000C2B300000000000000007B
:101EF20000000000AF80D2B3000000000000D2B2A8
:101F0200E4FCFDFEE5492FF549EE3548F548ED358F
:101F120047F547EC3546F546EBB54304EA696007F9
:101F22000AEA70A60B80A3AF49AE48AD47AC46782B
:101F320010120A12AB07AF49AE48AD47AC4678085B
:101F4200120A128F44E549FFE48F45AF03FE125592
:101F5200A7125787AF447E001255A7125787AF4585
:051F62007E000255A7FE
:1041BB00754DAA125A0A7F017E00125202C2B5C275
:1041CB00D97F017E001252027590D00000000000D2
:1041DB0000C2B27590500000000000007590D0E452
:1041EB00FFFE0000000000000FBF00010EEF646433
:1041FB004E70EFD2B27590FFE4FEFF00000000009E
:10420B00000FBF00010EEF64284E70EFE4F5A0F530
:10421B0080D2DBC2DB7580FF7590C0000000000010
:10422B0000C2B20000C2B3000000000000AF80D299
:0C423B00B30000D2B2EF6002F54DAF4DB1
:014247002254
:102F4D007540AAE4F541F542125A0A7F017E00123E
:102F5D005202C2B57F0A7E00125202C2D97F017E93
:102F6D00001252027834E6F53C08E6F53D7837E676
:102F7D00F53E08E6F53F853CA0853D80D2DBC2DB02
:102F8D007580FF7590C0000000000000C2B2000007
:102F9D00C2B300000000000085803BD2B30000D218
:102FAD00B2AF3B7E001255A70542E54270020541C6
:102FBD00B40029E541B402241257878F40E53B65E3
:102FCD0040600D7F557E001255A7153C153C8007BE
:102FDD007FAA7E001255A7E4F541F542E53CB53ECA
:102FED0006E53D653F600A053DE53D7089053C8080
:012FFD00854E
:012FFE0022B0
:1048A600125A0A7F017E00125202C2B590F002E44B
:1048B60093F54E25E0F54EC2D97F017E00125202D5
:1048C6007590C8000075A0010000E4F5800000D2D4
:1048D600DBC2DB0000C2B200007590480000759094
:1048E600C800007F0AFE125202D2B275A001000073
:1048F600854E800000D2DBC2DB7590CBC2B20000D1
:1049060075904B00007590CB0000E4FFFE000000A0
:104916000000000FBF00010EEF64294E70EF00008B
:02492600D2B20B
:01492800226C
:10580500125A0A7F017E00125202C2B5C2D97F0127
:105815007E00125202E4F5A0F580D2DBC2DB758072
:10582500FF7590D0C2B2C2B30000000000007590B1
:0A58350050AF807590D0D2B3D2B20C
:01583F002246
:1038F600125A0A7F017E00125202C2B5C2D97F0A4D
:103906007E001252027580FF90F004E493FDA3E45A
:1039160093FC90F007E493F54FA3E493F975BF0881
:10392600EDFEEC7A002400FFEA3E8F82F583E07517
:10393600BF028DA08C80D2DBC2DB7580FF0000F554
:10394600807590C0D2B3C2B2000075904000007579
:1039560090C0E4FFFE0000000000000FBF00010E53
:10396600EF64054E70EFD2B2EDB54F04EC69600717
:103976000CEC70A90D80A6E4FEFF0000000000001C
:0B3986000FBF00010EEF64284E70EF31
:013991002213
:10447600752FAA125A0A7F017E00125202C2B57F18
:104486000A7E00125202C2D97F017E0012520290A9
:10449600F004E493FDA3E493FC90F007E493F52D78
:1044A600A3E493F52E8DA08C80D2DBC2DB7580FF52
:1044B6007590C0000000000000C2B20000C2B30048
:1044C6000000000000A980D2B30000D2B275BF0878
:1044D600EDFEEC7A002400FFEA3E8F82F583E0755C
:1044E600BF02696002892FEDB52D05EC652E6007C8
:0944F6000CEC70B10D80AEAF2F8B
:0144FF00229A
:10169C00E4F52AF529F528F527F52BF52C125A0A2D
:1016AC00C2B57834E6F52108E6F5227837E6F5235D
:1016BC0008E6F52475F65575F6AA75F65575BF0C42
:1016CC00E4F5F475F7A275F7A205F405F4052CE51D
:1016DC002C7002052B6480452B70E81257878521EE
:1016EC00F48522F58FF675F7A0E521FE7C00E42544
:1016FC0022FFEC3E8F82F583E0FFE4FDFEE52A2F0E
:10170C00F52AEE3529F529ED3528F528EC3527F5A0
:10171C0027E521B52306E5226524600A0522E5228A
:10172C0070B9052180B575BF02AF2AAE29AD28ACC2
:10173C00277810120A12AB07AF2AAE29AD28AC27B6
:10174C007808120A128F25E52AFFE48F26AF03FED4
:10175C001255A7125787AF257E001255A71257872F
:10176C00783AA6077B007A007930751B0BE4FD7F75
:0B177C00F01254C4AF267E000255A7F7
:1049A9007830E614601614602814603A14604A24BA
:1049B900FE605D24067063123D27801F124DF18F42
:1049C900087E001255A7D2B5E508B4AA0280268050
:1049D90049120F2C7F017E001252027FAA7E00121B
:1049E90055A7D2B58024121F671257878F08D2B5F1
:1049F900E508B4AA028013802112479F8F087E0020
:104A09001255A7D2B5E508B4AA04C2B68009800A2E
:0F4A1900122B04C2B6D2B5025A49C2B41259A028
:014A2800226B
:103D2700125A0A7F017E00125202C2B5D296C2B25F
:103D3700D2B3C290C291C29275A055758055D2DB9D
:103D4700C2DB7580AAC2970000D29775A02A75803A
:103D5700AAD2DBC2DB758055C2970000D29775A047
:103D670055758055D2DBC2DB758080C2970000D2C3
:103D77009775A055758055D2DBC2DB7580AAC297AF
:103D87000000D29775A02A7580AAD2DBC2DB7580A6
:103D970055C2970000D29775A055758055D2DBC2E2
:103DA700DB758010C2970000D2977580FFC2B330D1
:053DB70087FDD2B322DC
:104DF100125A0A7F017E00125202C2B57F0A7E005A
:104E01001252027590FF7833E6FF08E6FE08E6FDD0
:104E110008E6F50908E6F908E6FBEF139290EFA220
:104E2100E19291A2E292928EA08D80D2DBC2DB75DB
:104E310080FFC2B2C2B3AC80D2B3D2B2ECF4600391
:104E41007F5522EFB5090BEEB50107EDB503037FE1
:0D4E5100AA220DED70C40EEE70C00F80BDE2
:100F2C00125A0A7F017E00125202C2B57F047E0063
:100F3C00125202C2D9D2DA7F0A7E00125202758096
:100F4C00FF7833E6F50908E6F50A08E6F50B08E63E
:100F5C00F50C08E6F50D08E6F50E125787D296C289
:100F6C00B2D2B3C290C291C29275A055758055D2BF
:100F7C00DBC2DB7580AAC2970000D29775A02A75D8
:100F8C0080AAD2DBC2DB758055C2970000D2977560
:100F9C00A055758055D2DBC2DB7580A0C2970000CE
:100FAC00D297E509139290E509A2E19291A2E292FF
:100FBC0092850AA0850B80D2DBC2DB8F80C29700A2
:100FCC0000D297E509139290E509A2E19291A2E271
:100FDC009292850AA0850B80D2DBC2DB7580FFC2A2
:100FEC00B2C2B3AE80D2B3D2B2EFB506D6E509B574
:100FFC000C0BE50AB50D06E50B650E6017050BE548
:10100C000B6003020F66050AE50A6003020F660512
:04101C0009020F6650
:0110200022AD
:101F6700E4F511F510F50FF50E125A0A7F017E0000
:101F7700125202C2B57F0A7E001252027590FF7894
:101F870033E6FB08E6F908E6FA08E6F50908E6F598
:101F97000A08E6F50BEB139290EBA2E19291A2E20D
:101FA700929289A08A80D2DBC2DB7580FFC2B2C25F
:101FB700B3AF80D2B3D2B2E4FCFDFEE5112FF51129
:101FC700EE3510F510ED350FF50FEC350EF50EEB80
:101FD700B50909E9B50A05EA650B600B0AEA70B5A8
:101FE70009E970B10B80AEAF11AE10AD0FAC0E7832
:101FF70010120A12AB07AF11AE10AD0FAC0E780876
:10200700120A128F0CE511FFE48F0DAF03FE125574
:10201700A71257877F017E00125202AF0C7E001273
:1020270055A71257877F017E00125202AF0D7E001F
:032037000255A7A8
:10479F00125A0A7F0A7E00125202C2B5C2D97F0A8C
:1047AF007E001252027590DB000000000000000036
:1047BF00C2B2E4FFFE0000000000000FBF00010EB8
:1047CF00EF64324E70EFD2B2000000000000D2D979
:1047DF007590FFE4F5A0F580D2DBC2DB7580FF7525
:1047EF0090F80000C2B2C2B3AD800000000000001C
:1047FF00D2B3D2B2ED60037F5522E4FEFF0000007A
:10480F000000000FBF00010EEF64284E70EF75908F
:03481F00FF7FAA6E
:014822002273
:102B04007510AAE4F511F512125A0A7F017E00121B
:102B14005202C2B57F0A7E001252027590FF7833CA
:102B2400E6F50A08E6F50B08E6F50C08E6F50D08E7
:102B3400E6F50E08E6F50FE50A139290E50AA2E120
:102B44009291A2E29292850BA0850C80D2DBC2DB2B
:102B54007580FFC2B2C2B3858009D2B3D2B2AF09C5
:102B64007E001255A70512E51270020511B4002962
:102B7400E511B402241257878F10E5096510600D22
:102B84007F557E001255A7150B150B80077FAA7E73
:102B9400001255A7E4F511F512E50AB50D0BE50B86
:102BA400B50E06E50C650F6011050CE50C70880583
:0A2BB4000BE50B7082050A022B3BB3
:012BBE0022F4
:1059F80075BF02759850758920438780758DFFD2D1
:025A08008E22EC
:095A4000C2B4C2B5C2B6025A514B
:10596F00539040E4F580F5A0D2DBC2DBD2B2C2B2D5
:09597F00C2B3D2D9C2DAC29622E9
:105A0A001251F3D2B2D2B3D2B4D2B5D2B6D2D9D21B
:025A1A00DA228E
:10590300750AAA1251F3D2B2D2B3D2B4D2B5D2B677
:10591300D2D9D2DA7580FF000000000000AF80000A
:0A59230000EFF460037F55227FAA15
:01592D002257
:105A1C00E4F580F590F5A0C2B2C2B3D2B4D2B5D23F
:025A2C00B622A0
:1057C700E4F59075A0FFD2D9C2DA7F0AFE12520221
:1057D700759040D2D9D2DA7F017E0012520212515F
:1057E700FED2D9C2DA75A0AA00000000000075A099
:0E57F70055D2B4D2B5D2B67580FF75A0FF2290
:0255A700AB0750
:1055A900E4F519F518F517F516C2998B992099356F
:1055B900000000000000E5192401F519E43518F58B
:1055C90018E43517F517E43516F5167F407E0D7D7D
:1055D900037C00AB19AA18A917F8C3120A0170CDE8
:0555E9001259CE80C83C
:0155EE00229A
:10578700E4F519F518F517F51620982FE5192401F2
:10579700F519E43518F518E43517F517E43516F556
:1057A700167F407E0D7D037C00AB19AA18A917F858
:0F57B700C3120A0170D31259CE80CEC298AF9997
:0157C60022C0
:1059880020D80D7F1E7E0012520220D8F37F1122EC
:085998003098EDC298AF99228E
:0654C4008B188A19891AF9
:1054CA0075F65575F6AA75F65575BF068FF48DF5FE
:1054DA0075F78275F782E47854F67854E6FFC39537
:1054EA001B5020AB18AA19A91A8F827583001209BA
:1054FA004FF5F675F78005F5E5F5700205F4785471
:06550A000680D775BF0208
:015510002278
:0F51F300D2967580FF7590FF75A0FF7F0A7E0032
:045202008E168F175E
:10520600E4FBFA4389017518F87519CDC3EB9517B8
:10521600E5166480F8EA648098502DAE18AF197CC4
:10522600017D0012097C8F8CAE18AF197C017D00C0
:1052360012097C8D8AD28C208D030080FAC28CC222
:0B5246008D0BBB00010A80C45389FEE1
:01525100223A
:105A2E00125A0A7F221255A7125988BF2203125A00
:015A3E004027
:015A3F002244
:104E5E0090F001E493FF120A254EBC014EBC024EA7
:104E6E00BC044EBF054EC2064EA7404EA7414EA7EC
:104E7E00424EB0504EB0514EB6524EB3534EC55434
:104E8E004EAA704EB9744EAA784EAA804EAD814E7F
:104E9E00AA844EAA8800004EC80205260207FC020C
:104EAE000D020200030201BB0206A00203730249B7
:0C4EBE00A9020E19020AA002371FC2B49C
:014ECA0022C5
:1059CE0075971E7597E1759FA07597E175971E786F
:0559DE0039765580FE42
:085A4900C2D81251FED2D8228E
:1059A000900000C2D81251FED2D81251FEA3E58257
:0659B000640B458370ED5D
:0159B60022CE
:1059B700900000C2D81251FED2D81251FEA3E58240
:0659C7006433458370ED1E
:0159CD0022B7
:10595000900000C2D87F287E00125202D2D87F1455
:0E5960007E00125202A3E5826402458370E5C8
:01596E002216
:035A510002FE0052
:030000000259E3BF
:1059E300E5BF5480700975BF02787FE4F6D8FD7572
:0559F300815402243F75
:100E19007830E6120A250E3E000E45010E5B020EE1
:100E290069030E7D040E93050EA7060EB0070EC0CA
:100E39001100000F261253C17F1E801B124F378FDE
:100E4900087E001255A7D2B5E508B4AA028064024B
:100E59000F2612409D7F017E001252027FAA804C0C
:100E69001222A71257878F08D2B5E508B4AA0280C3
:100E790042020F2612195D8F087E001255A7D2B5BE
:100E8900E508B4AA02802C020F2612178712578789
:100E99008F08D2B5E508B4AA028018020F261228D5
:100EA90017C2B6D2B5807312546F8F087E001255DF
:100EB900A7D2B5C2B6806390F00AE493F50930E091
:100EC9000A1253C17F1E7E00125202E50930E11851
:100ED900124F378F08E50864AA60028035C2B67FD1
:100EE9001E7E00125202D2B6E50930E2031235DF46
:100EF900E50930E30D124AA78F08E50864AA6002E4
:100F09008010E50930E40F12195D8F08E50864AA1D
:100F19006004D2B58007D2B5C2B6025A49C2B4122A
:020F290059A0CD
:010F2B0022A3
:1053C100125A1C7F017E00125202C2B5E4F590C24E
:1053D100B2D2B37590407F0AFE1252027590CA0094
:1053E100000000000000007590CB7F647E00125227
:1053F100027590C9E4FFFE0000000000000FBF002D
:10540100010EEF64144E70EF759040000000000033
:0654110000E4F59000002C
:015417002272
:1052AF00125A1C7F017E00125202C2B5E4F590C261
:1052BF00B2D2B3F5507590407F0AFE12520285505C
:1052CF00A0E4F580D2DBC2DB7590C20000000000C5
:1052DF000000007590C37F0AFE1252027590C10044
:1052EF000000000000000075904000000000055015
:0B52FF000550E55070C8E4F590000079
:01530A002280
:104F3700125A1C7F017E00125202C2B5E4F590C2DC
:104F4700B2D2B37590407F0AFE12520290F004E489
:104F570093FFA3E493FE90F007E493FDA3E493FC8F
:104F67008FA08E80D2DBC2DB7580FF7590C07590F5
:104F7700F0D2B2C2B3AB80D2B3C2B27590C0EBF479
:104F870060037F5522EFB50507EEB504037FAA221C
:074F97000EEE70CC0F80C983
:10409D00125A1C7F017E00125202C2B5E4F590C285
:1040AD00B2D2B37590407F0AFE1252027580FF9016
:1040BD00F004E493F50AA3E493F50B750CFF750D6D
:1040CD00FF7590C40000850AA0850B80D2DBC2DB92
:1040DD007580FF7590C500001257878F807590E52C
:1040ED00E4FFFE0000000000000FBF00010EEF64B2
:1040FD00054E70EF7590C500007590C10000000071
:10410D000000759040E50AB50C06E50B650D600ADB
:0F411D00050BE50B70AB050A80A7E4F5900000D9
:01412C002270
:1022A700E4F510F50FF50EF50D125A1C7F017E00AF
:1022B700125202C2B5E4F590C2B2D2B37590407F14
:1022C7000AFE12520290F004E493FBA3E493FA90FF
:1022D700F007E493F50AA3E493F98BA08A80D2DB95
:1022E700C2DB7580FF7590C07590F0D2B2C2B3AFF4
:1022F70080D2B3C2B27590C0E4FCFDFEE5102FF5A5
:1023070010EE350FF50FED350EF50EEC350DF50D1D
:10231700EBB50A04EA6960070AEA70BE0B80BB7571
:102327009040000000000000AF10AE0FAD0EAC0DE6
:102337007810120A12AB07AF10AE0FAD0EAC0D78C6
:1023470008120A128F0BE510FFE48F0CAF03FE1281
:1023570055A7125787AF0B7E001255A7125787AFA5
:0B2367000C7E001255A7E4F59000006A
:012372002248
:10195D00125A1C7F0A7E00125202C2B5E4F590C2E3
:10196D00B2D2B37590407F0AFE125202E4F5A0F593
:10197D0080D2DBC2DB7580FF7590C07590F0D2B25E
:10198D00C2B385800A7480250AF50AD2B3C2B27536
:10199D0090C00000000000000000000000007590E5
:1019AD00400000000000000000C2B2D2B3759040AC
:1019BD007F0A7E001252027580FF7590C40000E40C
:1019CD00F5A0F580D2DBC2DB7580FF7590C50000F8
:1019DD00850A807590E5FFFE0000000000000FBF36
:1019ED0000010EEF64054E70EF7590C50000759007
:1019FD00C1000000000000759040000000000000D4
:101A0D000000E4F5A0F580D2DBC2DB7580FF759098
:101A1D00C07590F0D2B2C2B385800AC2B3C2B2759E
:101A2D0090C0E50A60037F552275904000000000CC
:091A3D000000E4F59000007FAA0E
:011A4600227D
:10281700E4F50FF510125A1C7F017E00125202C216
:10282700B5E4F590C2B2D2B37590407F0AFE12525A
:10283700027834E6F50B08E6F50C7837E6F50D086F
:10284700E6F50E850BA0850C80D2DBC2DB7580FF19
:102857007590C07590F0D2B2C2B385800AD2B3C268
:10286700B27590C0AF0A7E001255A70000000000A5
:10287700000000000000000510E5107002050FB40D
:102887000026E50FB40221125787E50A6F600D7F16
:10289700557E001255A7150B150B80077FAA7E00E2
:1028A7001255A7E4F50FF510E50BB50D06E50C6518
:1028B7000E600A050CE50C708A050B808675904042
:0B28C700000000000000E4F59000009D
:0128D20022E3
:104C9600125A1C7F017E00125202C2B590F002E445
:104CA60093F5512480F551E4F590C2B2D2B37590D4
:104CB600407F0AFE1252027580FF7590C40000E420
:104CC600F5A0F580D2DBC2DB7580FF7590C50000CC
:104CD6008551807590E5FFFE0000000000000FBFC3
:104CE60000010EEF64054E70EF7590C500007590DB
:104CF600C1000000000000759040000000000000A8
:054D0600E4F59000003F
:014D0B002285
:10546F00125A1C7F017E00125202C2B5E4F590C29F
:10547F00B2D2B37590407F0AFE125202E4F5A0F546
:10548F0080D2DBC2DB7580FF7590C07590F0D2B211
:10549F00C2B3AF80D2B3C2B27590C000000000009B
:1054AF0000000000000000759040000000000000A8
:0454BF00F590000064
:0154C30022C6
:10178700E4F513F512F511F510F514F515125A0ACB
:10179700C2B57834E6F50A08E6F50B7837E6F50CB6
:1017A70008E6F50D75F65575F6AA75F65575BF0C6D
:1017B700E4F5F475F7A275F7A205F405F40515E548
:1017C70015700205146480451470E8850AF4850BCA
:1017D700F51257878FF675F7A0E50AFE7C00E4251A
:1017E7000BFFEC3E8F82F583E0FFE4FDFEE5132F50
:1017F700F513EE3512F512ED3511F511EC3510F53F
:1018070010E50AB50C06E50B650D600A050BE50B3F
:1018170070B9050A80B575BF02AF13AE12AD11AC32
:10182700107810120A12AB07AF13AE12AD11AC103D
:101837007808120A128F0EE513FFE48F0FAF03FE2D
:101847001255A7125787AF0E7E001255A71257875A
:10185700783AA6077B007A007930751B0BE4FD7F89
:0B186700F01254C4AF0F7E000255A722
:1035DF00125A0A7F017E00125202C2B57F047E008A
:1035EF00125202C2D9D2DA7F0A7E001252027580BD
:1035FF00FF90F004E493FDA3E493FC90F007E493B1
:10360F00F50AA3E493F98DA08C80D2DBC2DB758021
:10361F00FF000075BF08EDFEEC7A002400FFEA3EC4
:10362F008F82F583E0F58075BF027590570000C259
:10363F00B2000075905FE4FFFE0000000000000F75
:10364F00BF00010EEF64054E70EFD2B2EDB50A0464
:10365F00EC6960070CEC70AE0D80ABE4FEFF000070
:0F366F00000000000FBF00010EEF64284E70EF47
:01367E002229
:104AA700750CAA125A0A7F017E00125202C2B5D2B1
:104AB700D9D2DA7F0A7E001252027590FF90F00475
:104AC700E493FDA3E493FC90F007E493F50AA3E4D1
:104AD70093F50B8DA08C80D2DBC2DB7580FF7590C0
:104AE700807590E0D2B2D2B3A980759080C2B3C26C
:104AF700B275BF08EDFEEC7A002400FFEA3E8F8214
:104B0700F583E075BF026960037F5522EDB50A079B
:0E4B1700ECB50B037FAA220CEC70B80D80B534
:100AA0007830E6120A250AC5000ADB010AF2020BB9
:100AB0001B030B2F040B45050B59060B62070B722A
:100AC0001100000BD81254187F1E7E001252021221
:100AD00054187F1E7E00125202803C124F9E8F08D7
:100AE0007E001255A7D2B5E508B4AA03020B6E0228
:100AF0000BD8123BF8124C1F12530B8F087F017E4C
:100B00000012520290F002E4936508600A7F557E5D
:100B1000001255A7020BCD7FAA804C1223731257E7
:100B2000878F08D2B5E508B4AA028042020BD8121A
:100B300039928F087E001255A7D2B5E508B4AA02F3
:100B4000802C020BD81218721257878F08D2B5E585
:100B500008B4AA028018020BD8122C78C2B6D2B5FB
:100B6000807312530B8F087E001255A7D2B5C2B600
:100B7000806390F00AE493F50930E00A1254187F7C
:100B80001E7E00125202E50930E118124F9E8F08B6
:100B9000E50864AA60028035C2B67F1E7E0012524C
:100BA00002D2B6E50930E20312367FE50930E30DE3
:100BB000124B258F08E50864AA60028010E5093011
:100BC000E40F1239928F08E50864AA6004D2B58058
:0D0BD00007D2B5C2B6025A49C2B41259A0EC
:010BDD0022F5
:105418001257C77F017E00125202C2B5E4F590C24E
:10542800B2D2B37590407F0AFE1252027590CA003C
:10543800000000000000007590CB7F647E001252CF
:10544800027590C9E4FFFE0000000000000FBF00D5
:10545800010EEF64144E70EF7590400000000000DC
:0654680000E4F5900000D5
:01546E00221B
:105252001257C77F017E00125202C2B5E4F590C216
:10526200B2C2B3F5527590407F0AFE1252028552C5
:10527200A0E4F580D2DBC2DB7590C2000000000022
:105282000000007590C37F0AFE1252027590C100A1
:105292000000000000000075904000000000055270
:0C52A2000552E552B4FEC7E4F590000090
:0152AE0022DD
:104F9E001257C77F017E00125202C2B5E4F590C2CD
:104FAE00B2C2B37590407F0AFE12520290F004E432
:104FBE0093FFA3E493FE90F007E493FDA3E493FC28
:104FCE008FA08E80D2DBC2DB7580FF7590C075908E
:104FDE00F0D2B2C2B3AB80C2B3C2B27590C0EBF422
:104FEE0060037F5522EFB50507EEB504037FAA22B5
:074FFE000EEE70CC0F80C91C
:103BF8001257C77F017E00125202C2B5E4F590C287
:103C0800B2C2B37590407F0AFE1252027580FF90CF
:103C1800F004E493F50AA3E493F50B90F007E4931A
:103C2800F50CA3E493F50D7590C40000850AA085F2
:103C38000B80D2DBC2DB7580FF7590C50000125780
:103C4800878F807590E5E4FFFE0000000000000FFC
:103C5800BF00010EEF64084E70EF7590C500007547
:103C680090C10000759040E50AB50C06E50B650D9E
:103C7800600A050BE50B70AF050A80AB0000000079
:073C88000000E4F5900000CC
:013C8F002212
:10237300E4F510F50FF50EF50D1257C77F017E003A
:10238300125202C2B5E4F590C2B2C2B37590407F57
:102393000AFE12520290F004E493FBA3E493FA9032
:1023A300F007E493F50AA3E493F98BA08A80D2DBC8
:1023B300C2DB7580FF7590C07590F0D2B2C2B3AF27
:1023C30080C2B3C2B27590C0E4FCFDFEE5102FF5E8
:1023D30010EE350FF50FED350EF50EEC350DF50D51
:1023E300EBB50A04EA6960070AEA70BE0B80BB75A5
:1023F3009040000000000000AF10AE0FAD0EAC0D1A
:102403007810120A12AB07AF10AE0FAD0EAC0D78F9
:1024130008120A128F0BE510FFE48F0CAF03FE12B4
:1024230055A7125787AF0B7E001255A7125787AFD8
:0B2433000C7E001255A7E4F59000009D
:01243E00227B
:103992001257C77F0A7E00125202C2B5C2B2D2B318
:1039A2007590407F0A7E001252027580FF7590C4A6
:1039B2000000E4F5A0F580D2DBC2DB7580FF7590D4
:1039C200C5000075807F7590E5FFFE0000000000D5
:1039D200000FBF00010EEF64054E70EF7590C50039
:1039E200007590C1000000000000759040000000CA
:1039F2000000000000E4F5A0F580D2DBC2DB758098
:103A0200FF7590C07590F0D2B2C2B3AF80C2B3C29C
:103A1200B27590C0EF60037F5522759040000000A0
:0A3A2200000000E4F59000007FAA08
:013A2C002277
:102C7800E4F50FF5101257C77F017E00125202C209
:102C8800B5E4F590C2B2C2B37590407F0AFE125205
:102C980002E4F50BF50C7837E6F50D08E6F50E8538
:102CA8000BA0850C80D2DBC2DB7580FF7590C075E8
:102CB80090F0D2B2C2B385800AC2B3C2B27590C0D6
:102CC800AF0A7E001255A7000000000000000000B7
:102CD8000000000510E5107002050FB40026E50F8E
:102CE800B40221125787E50A6F600D7F557E0012E6
:102CF80055A7150B150B80077FAA7E001255A7E470
:102D0800F50FF510E50BB50D06E50C650E600A0527
:102D18000CE50C708A050B80867590400000000059
:072D28000000E4F59000003B
:012D2F002281
:104C1F001257C77F017E00125202C2B590F002E414
:104C2F0093F50A24E0F50AE4F590C2B2D2B3759079
:104C3F00407F0AFE1252027580FF7590C40000E497
:104C4F00F5A0758001D2DBC2DB7580FF7590C500C2
:104C5F0000850A807590E5FFFE0000000000000F40
:104C6F00BF00010EEF64054E70EF7590C500007523
:104C7F0090C100000000000075904000000000008F
:064C8F0000E4F5900000B6
:014C950022FC
:10530B001257C77F017E00125202C2B5E4F590C25C
:10531B00B2D2B37590407F0AFE125202E4F5A0752B
:10532B008001D2DBC2DB7580FF7590C07590F0D227
:10533B00B2D2B3AF8074202FFFD2B3C2B27590C07C
:10534B00000000000000000000000000759040000D
:0A535B000000000000E4F5900000DF
:015365002225
:10187200E4F513F512F511F510F514F515125A0ADF
:10188200C2B57834E6F50A08E6F50B7837E6F50CCA
:1018920008E6F50D75F65575F6AA75F65575BF0C81
:1018A200E4F5F475F7A275F7A205F405F40515E55C
:1018B20015700205146480451470E8850AF4850BDE
:1018C200F51257878FF675F7A0E50AFE7C00E4252E
:1018D2000BFFEC3E8F82F583E0FFE4FDFEE5132F64
:1018E200F513EE3512F512ED3511F511EC3510F553
:1018F20010E50AB50C06E50B650D600A050BE50B54
:1019020070B9050A80B575BF02AF13AE12AD11AC46
:10191200107810120A12AB07AF13AE12AD11AC1051
:101922007808120A128F0EE513FFE48F0FAF03FE41
:101932001255A7125787AF0E7E001255A71257876E
:10194200783AA6077B007A007930751B0BE4FD7F9D
:0B195200F01254C4AF0F7E000255A736
:10367F00125A0A7F017E00125202C2B57F047E00E9
:10368F00125202C2D9D2DA7F0A7E0012520275801C
:10369F00FF90F004E493FDA3E493FC90F007E49310
:1036AF00F50AA3E493F98DA08C80D2DBC2DB758081
:1036BF00FF000075BF08EDFEEC7A002400FFEA3E24
:1036CF008F82F583E0F58075BF027590570000C2B9
:1036DF00B2000075905FE4FFFE0000000000000FD5
:1036EF00BF00010EEF64054E70EFD2B2EDB50A04C4
:1036FF00EC6960070CEC70AE0D80ABE4FEFF0000D0
:0F370F00000000000FBF00010EEF64284E70EFA6
:01371E002288
:104B2500750CAA125A0A7F017E00125202C2B5D232
:104B3500D9D2DA7F0A7E001252027590FF90F004F6
:104B4500E493FDA3E493FC90F007E493F50AA3E452
:104B550093F50B8DA08C80D2DBC2DB7580FF759041
:104B6500807590E0D2B2D2B3A980759080C2B3C2ED
:104B7500B275BF08EDFEEC7A002400FFEA3E8F8295
:104B8500F583E075BF026960037F5522EDB50A071D
:0E4B9500ECB50B037FAA220CEC70B80D80B5B6
:1001BB007830E6120A2501E0000214010230020237
:1001CB006703027B0402910502A50602AE0702BF7C
:1001DB00110000036D125636E4FF1250D41257056E
:1001EB008F08E508600BD2B5C2B41259A07F5580B9
:1001FB00661258A57F1E7E001252021258A5D2B568
:10020B00C2B6125A497FAA804E12400C8F08D2B543
:10021B00E508B4AA07C2B6125A498005C2B41259EE
:10022B00A0AF088032122FFF1256361250CE125743
:10023B00058F087F017E0012520290F002E4936555
:10024B0008600BD2B5C2B41259A07F558009D2B544
:10025B00C2B6125A497FAA7E000255A7121A47123C
:10026B0057878F08D2B5E508B4AA02804202036D06
:10027B00123DBC8F087E001255A7D2B5E508B4AA73
:10028B0002802C02036D1211131257878F08D2B5FF
:10029B00E508B4AA02801802036D1221DAC2B6D2A5
:1002AB00B5800E1257058F087E001255A7D2B5C226
:1002BB00B6025A4990F00AE493F50930E028125639
:1002CB0036E4FF1250D41257058F08E5086003027D
:1002DB00035F1258A57F1E7E001252021258A5D240
:1002EB00B5C2B6125A49E50930E11412400C8F0819
:1002FB00E50864AA6002805CD2B5C2B6125A49E521
:10030B000930E227122D301256361250CE125705F5
:10031B008F087F017E0012520290F002E493650871
:10032B0060028030D2B5C2B6125A49E50930E314E7
:10033B001233FD8F08E50864AA60028017D2B5C29C
:10034B00B6125A49E50930E416123DBC8F08E50890
:10035B0064AA6004D2B5800AD2B5C2B6125A490259
:07036B00596FC2B41259A042
:010372002268
:1058A500125A0A7F017E00125202C2B5D2D9C2DA5B
:1058B5007590F0C2B2000075907000007590F00010
:0F58C500007FB07E04125202D2B2D2D9D2DA22C0
:10400C00125A0A7F017E00125202C2B57F0A7E004C
:10401C00125202D2D9C2DA7F017E0012520290F003
:10402C0004E493FFA3E493FE90F007E493FDA3E470
:10403C0093FC8FA0EE54C0C413135403FBEE543FF7
:10404C00F580D2DBC2DB7580FFEB44C0F59000003D
:10405C0000000000C2B2000000000000C2B300006B
:10406C0000000000AB80D2B3000000000000D2B210
:10407C00EBF46007D2D9D2DA7F5522EFB5050BEEFF
:10408C00B50407D2D9D2DA7FAA220EEE70A40F8023
:01409C00A182
:102FFF00125A0A7F017E00125202C2B5D2D9C2DA2A
:10300F007F0A7E001252027580FF90F004E493F560
:10301F000AA3E493F50B90F007E493F50CA3E49364
:10302F00F50D850AA0E50B54C0FFC413135403F527
:10303F000EE50B543FF580D2DBC2DB7580FF00003D
:10304F001257878F80E50E44C0FFF590D2B3C2B2FE
:10305F000000E50E4440F59000008F90E4FFFE0065
:10306F0000000000000FBF00010EEF64054E70EF6F
:10307F00D2B2E50AB50C0BE50BB50D06D2D9D2DAF3
:10308F00800A050BE50B709A050A8096E4FEFF0097
:10309F0000000000000FBF00010EEF64284E70EF1C
:0130AF0022FE
:101A4700E4F511F510F50FF50E125A0A7F017E0025
:101A5700125202C2B57F0A7E00125202D2D9C2DAEE
:101A67007F017E0012520290F004E493FBA3E493FB
:101A7700FA90F007E493F50AA3E493F98BA0EA54EC
:101A8700C0C413135403FFEA543FF580D2DBC2DB13
:101A97007580FFEF44C0F590000000000000C2B25F
:101AA7000000C2B3000000000000AF80D2B3000006
:101AB700D2B2E4FCFDFEE5112FF511EE3510F5105D
:101AC700ED350FF50FEC350EF50EEBB50A0AEAB555
:101AD7000106D2D9D2DA80070AEA70A00B809DAF3F
:101AE70011AE10AD0FAC0E7810120A128F0BAF119A
:101AF700AE10AD0FAC0E7808120A128F0CE511FF6D
:101B0700E48F0D7F0AFE125202AF0B7E001255A71B
:101B1700125787AF0C7E001255A7125787AF0D7E5D
:041B2700000255A7BC
:103DBC00750AAA125A0A7F017E00125202C2B5D2AB
:103DCC00D9C2DA7F017E001252027590D00000C277
:103DDC00B275905000007590D0E4FFFE000000001A
:103DEC0000000FBF00010EEF64324E70EFD2B275BF
:103DFC0090FFE4FEFF0000000000000FBF00010E6A
:103E0C00EF64144E70EFE4F5A0C413135403FEE4F6
:103E1C00F580D2DBC2DB7580FFEE44C0F59000006C
:103E2C0000000000C2B20000C2B30000000000009D
:103E3C00AF80D2B30000D2B2D2D9D2DAEF60037F16
:043E4C0055227FAAD2
:013E5000224F
:1021DA00750FAAE4F510F511125A0A7F017E001252
:1021EA005202C2B57F0A7E00125202D2D9C2DA7FE7
:1021FA00017E001252027834E6F50B08E6F50C78F7
:10220A0037E6F50D08E6F50E850BA0E50C54C0C4BB
:10221A0013135403FFE50C543FF580D2DBC2DB7580
:10222A0080FFEF44C0F590000000000000C2B20039
:10223A0000C2B300000000000085800AD2B300008B
:10224A00D2B2AF0A7E001255A70511E51170020538
:10225A0010B4002FE510B4022A1257878F0FE50A2F
:10226A00650F600D7F557E001255A7150B150B8063
:10227A00077FAA7E001255A7E4F510F5117F14FE18
:10228A00125202E50BB50D06E50C650E600E050C43
:0C229A00E50C6003022212050B02221268
:0122A6002215
:10563600125A0A7F017E00125202C2B5D2D9C2DACC
:105646007F017E001252027590C8000075A001000D
:1056560000E4F5800000D2DBC2DB0000C2B200002D
:1056660075904800007590C800007F0AFE1252022D
:07567600D2B2D2D9D2DA2230
:0650CE0090F002E493FFE4
:0250D4008F0A41
:1050D600125A0A7F017E00125202C2B5E50A25E085
:1050E600F50AD2D9C2DA7F017E0012520275A001FA
:1050F6000000E50A44C0F5800000D2DBC2DB7590F3
:10510600C8C2B2000075904800007590C80000E45F
:10511600FFFE0000000000000FBF00010EEF642933
:0B5126004E70EF0000D2B2D2D9D2DAF6
:01513100225B
:10570500125A0A7F017E00125202C2B5D2D9C2DAFC
:105715007F017E00125202E4F5A0F580D2DBC2DBE8
:105725007580FF7590D0C2B2C2B3000000000000C2
:10573500759050AF807590D0D2B3D2B2D2D9D2DAAB
:015745002241
:102D3000125A0A7F017E00125202C2B5D2D9C2DAFB
:102D40007F0A7E001252027580FF90F004E493FD2A
:102D5000A3E493FC90F007E493F50AA3E493F50B46
:102D60008DA0EC54C0C413135403F9EC543FF58008
:102D7000D2DBC2DB7580FF000075BF08EDFEEC7A88
:102D8000002400FFEA3E8F82F583E0F58075BF02E4
:102D9000E944C0FFF590D2B3C2B20000E94440F567
:102DA0009000008F90E4FFFE0000000000000FBFC5
:102DB00000010EEF64054E70EFD2B2EDB50A0AECD9
:102DC000B50B06D2D9D2DA80070CEC70930D809047
:102DD000E4FEFF0000000000000FBF00010EEF64E2
:042DE000284E70EF1A
:012DE40022CC
:1033FD00750CAA125A0A7F017E00125202C2B57FC5
:10340D000A7E00125202D2D9C2DA7F017E00125218
:10341D000290F004E493FDA3E493FC90F007E49391
:10342D00F50AA3E493F50B8DA0EC54C0C41313540B
:10343D0003FFEC543FF580D2DBC2DB7580FFEF4418
:10344D00C0F590000000000000C2B20000C2B30041
:10345D000000000000A980D2B30000D2B275BF08F1
:10346D00EDFEEC7A002400FFEA3E8F82F583E075D5
:10347D00BF02696007D2D9D2DA7F5522EDB50A0BAA
:10348D00ECB50B07D2D9D2DA7FAA220CEC70980DCD
:02349D00809518
:10111300E4F513F512F511F510F514F515125A0A45
:10112300C2B57834E6F50A08E6F50B7837E6F50C30
:1011330008E6F50D75F65575F6AA75F65575BF0CE7
:10114300E4F5F475F7A275F7A205F405F40515E5C2
:1011530015700205146480451470E8850AF4850B44
:10116300F51257878FF675F7A0E50AFE7C00E42594
:101173000BFFEC3E8F82F583E0FFE4FDFEE5132FCA
:10118300F513EE3512F512ED3511F511EC3510F5B9
:1011930010E50AB50C06E50B650D600A050BE50BBA
:1011A30070B9050A80B575BF027F0A7E001252022C
:1011B300AF13AE12AD11AC107810120A12AB07AF19
:1011C30013AE12AD11AC107808120A128F0EE5138C
:1011D300FFE48F0FAF03FE1255A7125787AF0E7EA2
:1011E300001255A7125787783AA6077B007A007931
:1011F30030751B0BE4FD7FF01254C4AF0F7E000269
:0212030055A7ED
:10371F007830E6120A25374400375C0137780237D4
:10372F008903378E0437A60537AB0637B00737B591
:10373F0011000037B81258D47F1E7E0012520212A9
:10374F0058D4D2B5C2B6125A497FAA8028124D0C4E
:10375F008F08D2B5E508B4AA07C2B6125A49800538
:10376F00C2B41259A0AF08800C125A57D2B5C2B4C6
:10377F001259A07F557E000255A7125A58802A125F
:10378F0043608F087E001255A7D2B5E508B4AA058D
:10379F00C2B6025A498012125A5B800D125A5980D2
:0E37AF0008125746800302596FC2B41259A087
:0137BD0022E9
:1058D400125A0A7F017E00125202C2B5D2D9C2DA2C
:1058E4007590F0C2B2000075907000007590F000E1
:0F58F400007FB07E04125202D2B2D2D9D2DA2291
:104D0C00125A0A7F017E00125202C2B57F0A7E003F
:104D1C00125202D2D9C2DA7F017E0012520290F0F6
:104D2C0004E493FFA3E493FE90F007E493FDA3E463
:104D3C0093F5098FA08E80D2DBC2DB7580FF759056
:104D4C00C0000000000000C2B2000000000000C261
:104D5C00B3000000000000AC80D2B30000000000E3
:104D6C0000D2B2ECF460037F55227EFF0FEFB50545
:034D7C00C27FAA49
:014D7F002211
:015A5700222C
:015A5800222B
:104360007509AA125A0A7F017E00125202C2B5D202
:10437000D9C2DA7F017E001252027590D00000C2CD
:10438000B275905000007590D0E4FFFE0000000070
:1043900000000FBF00010EEF64324E70EFD2B27515
:1043A00090FFE4FEFF0000000000000FBF00010EC0
:1043B000EF64144E70EFE4F5A0F580D2DBC2DB753C
:1043C00080FF7590C0000000000000C2B20000C273
:1043D000B3000000000000AF80D2B30000D2B2D220
:0B43E000D9D2DAEF60037F55227FAADC
:0143EB0022AF
:015A5900222A
:10567D00125A0A7F017E00125202C2B5D2D9C2DA85
:10568D007F017E001252027590C8000075A00100C6
:10569D0000E4F5800000D2DBC2DB0000C2B20000E6
:1056AD0075904800007590C800007F0AFE125202E6
:0756BD00D2B2D2D9D2DA22E9
:025366008F5363
:10536800125A0A7F017E00125202C2B5E55325E0A7
:10537800F553D2D9C2DA7F017E0012520275A0011C
:1053880000008553800000D2DBC2DB7590CBC2B22F
:10539800000075904B00007590CB0000E4FFFE0004
:1053A80000000000000FBF00010EEF64294E70EFEF
:0853B8000000D2B2D2D9D2DA12
:0153C00022CA
:10574600125A0A7F017E00125202C2B5D2D9C2DABB
:105756007F017E00125202E4F5A0F580D2DBC2DBA7
:105766007580FF7590D0C2B2C2B300000000000081
:10577600759050AF807590D0D2B3D2B2D2D9D2DA6A
:015786002200
:015A5A002229
:035A54007F0022AE
:015A5B002228
:10094F00BB010CE58229F582E5833AF583E022505D
:10095F0006E92582F8E622BBFE06E92582F8E222A7
:0D096F00E58229F582E5833AF583E49322C1
:10097C00C2D5EC30E709B2D5E4C39DFDE49CFCEE96
:10098C0030E715B2D5E4C39FFFE49EFE120A4BC3B9
:10099C00E49DFDE49CFC8003120A4B30D507C3E4B4
:0609AC009FFFE49EFE2205
:1009B200E88FF0A4CC8BF0A42CFCE98EF0A42CFCE4
:1009C2008AF0EDA42CFCEA8EF0A4CDA8F08BF0A462
:1009D2002DCC3825F0FDE98FF0A42CCD35F0FCEBC1
:1009E2008EF0A4FEA9F0EB8FF0A4CFC5F02ECD3986
:0F09F200FEE43CFCEAA42DCE35F0FDE43CFC22F3
:100A0100EB9FF5F0EA9E42F0E99D42F0E89C45F04B
:010A110022C2
:100A1200E8600FECC313FCED13FDEE13FEEF13FFC2
:030A2200D8F122E6
:100A2500D083D082F8E4937012740193700DA3A360
:100A350093F8740193F5828883E473740293686074
:060A4500EFA3A3A380DF74
:100A4B00BC000BBE0029EF8DF084FFADF022E4CC8F
:100A5B00F875F008EF2FFFEE33FEEC33FCEE9DEC58
:100A6B00984005FCEE9DFE0FD5F0E9E4CEFD22ED9E
:100A7B00F8F5F0EE8420D21CFEADF075F008EF2FE8
:100A8B00FFED33FD4007985006D5F0F222C398FDD9
:050A9B000FD5F0EA2276
:00000001FF
